:1000000008308A00FC2B0000FF00030E8301A100D2
:100010007F08A0000A08A8008A01A00E0408A20018
:100020007708A3007808A4007908A5007A08A6003C
:100030007B08A700831383128B1E20280B193328FB
:10004000220884002308F7002408F8002508F90096
:100050002608FA002708FB0028088A00210E8300E2
:10006000FF0E7F0E09008A11E9290A108A100A1171
:100070008207733431346A3429343F343E343C349B
:100080003834303420342134233427342F340134AD
:100090002A340134313468344C3456340634113443
:1000A00015340934023414340B34103404341E343F
:1000B0000D341234073405340F3416341B340A342B
:1000C000083403340C3418340E3419341D3413340A
:1000D0000A108A100A1182072034743469346D348E
:1000E00065342034283425346C34753429343A345A
:1000F000203400340A108A100A1182072034743424
:100100006F346E3465342034283425346C347534BF
:1001100029343A34203400340A108A100A11820734
:1001200020344D3473346734203428342534533428
:1001300029343A34203400340A108A100A11820714
:100140000D340A344134753474346F3420344334FC
:10015000573420344934443420342834253443344B
:1001600029343A34203400340A108A100A118207E4
:100170000D340A34433457342034533470346534E6
:1001800065346434203428342534553429343A34E1
:10019000203400340A108A100A1182070D340A3400
:1001A00049344434203461347534643469346F34F0
:1001B00000340A108A100A1182070D340A345234AE
:1001C0006534703465346134743465347234203489
:1001D0006D346F346434653420342834253443342A
:1001E00029343A34203400340A108A100A11FB3EB4
:1001F00003188A0A82000D340A3443346F3475348C
:100200007234743465347334793420346234653430
:100210006534703400340A148A100A1182070D34D0
:100220000A3443346F34753472347434653473343F
:100230007934203462346534653470342034643465
:1002400065346C346134793400340A148A100A112C
:1002500082070D340A3443346F3475347234743485
:1002600065347334793420346234653465347034E1
:1002700020346D3475346C3474342034283425348F
:10028000753429343A34203400340A148A100A119F
:1002900082070D340A3442346534613463346F3478
:1002A0006E3400340A148A100A1182070D340A349D
:1002B0005034543454342034683461346E346734E8
:1002C00000340A148A100A1182070D340A3450349B
:1002D0005434543420346D346134783400340A1486
:1002E0008A100A1182070D340A3449344434003428
:1002F0000A148A100A1182070D340A3459346534FD
:100300006C346C346F34773400340A148A100A1158
:1003100082070D340A3442346C3469346E346B34E1
:1003200000340A148A100A1182070D340A34533437
:1003300050344134433445342034773469346C3498
:100340006C342034643465346C346534743465340E
:10035000203449344434203473347434723469346E
:100360006E3467342E340D340A3449344434003446
:100370000A148A100A1182070D340A3441346C348D
:100380007434653472346E346134743465340034DA
:100390000A148A100A1182070A340D340A344E34C2
:1003A00030345834413453342034493444342D34B7
:1003B0004F342D344D346134743469346334203413
:1003C0005634253475342E34253475340A340D34BE
:1003D000003410300317A707003003180130A807B6
:1003E000003003180130A907A908031D092A2808AD
:1003F0000E3C0318A82AFF3A031D092A2708413C8E
:100400000318A82AFF3A031D092A2608403C0318AE
:10041000A82A4030A6024230031C4330A7020F3006
:10042000031C1030A8020030031C0130A902031382
:100430006F08593C031D202A0317AA1F302A0313F3
:10044000F508031D262AF60803192E2A0317AB10F8
:1004500075080319F603F503302A03130317AB14C9
:1004600083160313670F372A680F372A3A2AE70AD9
:100470000319E80AF10803193E2AF103831203174E
:10048000A408031D462AA50803194F2A24080319A6
:10049000A503A40324082504031D4F2A2A17831645
:1004A0000313610862040319662A76086202031CBA
:1004B000662A031D5F2A610875020318662A8312E3
:1004C00003172A14AA14AA118316031363086404D9
:1004D00003197B2A76086402031C7B2A031D742AF5
:1004E0006308750203187B2A831203172A14AA14BF
:1004F000AA158316031306128312061203172A1C69
:10050000872A83160313061283120616031783160F
:1005100003138612831286120317AA1C952A8316C8
:1005200003138612831286160317AA1DA82A2A1DF2
:10053000A12A8316031386128312861603172A1123
:10054000A82A8316031386128312861203172A150C
:1005500003130B118A112028031740088316031375
:100560009B009C131C141A08F80083120034031714
:100570003908C0000313AC220317BB017808BA0086
:1005800001303907BC00C0000313AC220030031750
:10059000BA070318BB0A7808BB073A08F8003B08FB
:1005A000F9000313003403174508F8014402031847
:1005B000DC2A4408F700E82AF7010830C600C40D19
:1005C000F70D450877020318F700F80DC60BDF2A70
:1005D00003130034780803174208C4006430C500D0
:1005E0000313D32277080317C20078083030031DA5
:1005F000002B43180B2BC3190B2B431A2030022B53
:10060000C3114312F807780803130C1A092B0317B8
:10061000042B990003174208C4000A30C5000313D5
:10062000D32277080317C20078083030031D1C2B33
:10063000C319252B431A2030F807780803130C1A26
:10064000232B03171E2B990003173030C2074208D3
:1006500003130C1A2D2B0317282B99000034453057
:100660008400831700080319442B0130F800F701B8
:10067000F70B382BF80B372B4A30F700F70B3E2BD4
:1006800000000000800B352B00340317BE013E082C
:10069000043C031C562B83160313650883120317AF
:1006A000C50003132F230317BE0A472B031300347F
:1006B000F801F901F701FA0103174B08031D632B39
:1006C0004A0803197D2B1030CC000310C80DC90D4A
:1006D000F70DFA0D4B087A02031D702B4A087702BA
:1006E000031C792B4A08F702031CFA034B08FA0291
:1006F0000314F80DF90DCC0B652B00000313003427
:100700000317C0080319E12B0430C900B030C8003A
:10071000CB0103136E080317CA000313582379088B
:100720008316E6007808E5000030F80006388312EA
:1007300092000317200883160313920083120317F5
:10074000210CC600200CC500C60CC50C3F30C605E8
:10075000C60CC50CC60CC50CC60C45080313950089
:100760000317C60C460C3039F70003131708CF39AE
:1007700077049700831686118312861583168510D9
:10078000831285140317C101400841020318D32BBB
:1007900083160313650883120317C50003132F2361
:1007A0000317C10AC42B8316031385108312851007
:1007B00083168615650883120317C50003132F23BC
:1007C00003170313003403173E0BE72BF32BBF0172
:1007D0000310BE0CBF0D0314BF0D3F08C000031370
:1007E0008023E32B0317BF013F08013C031C032CAC
:1007F00083160313650883120317C50003132F2301
:100800000317BF0AF42B03138A11242C03173C0887
:10081000203C031D0F2C03134523242C0317013008
:10082000BD003C082B3C0318202C3C085A3C031C00
:10083000202C2C303C0203133520F8000317BD0098
:100840003D08BE000313E32B003478080317390872
:10085000C4006430C5000313D32277080317B9001E
:1008600078083030031D3B2C3A18432CBA19432C1E
:100870003A1A20303D2CBA113A12F8077808BC0019
:100880000313062403173908C4000A30C5000313F4
:10089000D32277080317B90078083030031D542C91
:1008A000BA195A2C3A1A2030F8077808BC000313FA
:1008B000062403173030B9073908BC000313062497
:1008C000003483160510831205140317AA1A6D2C21
:1008D000AA162308A5002208A40003130034F70178
:1008E000F80103173F0803104018F707F70CF80C3E
:1008F000C018F707F70CF80C4019F707F70CF80CBD
:10090000C019F707F70CF80C401AF707F70CF80CAA
:10091000C01AF707F70CF80C401BF707F70CF80C98
:10092000C01BF707F70CF80C03138A11242D83164C
:100930000510831205100317AA12A501A4010313C1
:1009400000340317B9080319A82C3908BA00E22C9F
:10095000AB1CC12C83160313061483120618BD2C7E
:1009600094300317C0000313AC22F8080319BD2C00
:1009700094300317BA00C02C031314300317BA00C5
:10098000E22C5430C0000313AC22F8080319CD2C1C
:1009900054300317BA00E22C031383160614831293
:1009A0000618DF2C94300317C0000313AC22F8089C
:1009B0000319DF2C94300317BA00E22C0313143010
:1009C0000317BA002A14AA11AA10831603130617D4
:1009D0008312061BED2C0317E52C61240830031746
:1009E000BC00FA30C50003132F230317BC0BF12CF6
:1009F0003A08BA0ABC00C0000313AC2278080317F7
:100A0000BB00BB0803198B2D3B083A3C03190E2D84
:100A10003B08BC0003130624892D03173A08BC00C9
:100A2000BD013C08BC0ABF00C0000313AC2278081B
:100A30000317BE003E083A3C03192A2D3D08BF00AB
:100A40000A30C00003136F2C78080317BD00303044
:100A50003E02BD073E083A3C031D112D3D08F8003B
:100A60007808BB000030F800063803139200031723
:100A7000200883160313920083120317210CBD0074
:100A8000200CBC00BD0CBC0C3F30BD05BD0CBC0C2B
:100A9000BD0CBC0CBD0C3C08031395000317BD0C2A
:100AA0003D0C3039F70003131708CF39770497004E
:100AB000831686118312861583168510831285147A
:100AC00004300317BC00FA30C50003132F230317AB
:100AD000BC0B632DBB0303196F2D0313602D83160D
:100AE000031385108312851083168615831203174E
:100AF0003A08BA0ABC00C0000313AC2278080317F6
:100B0000BB003B083A3C0319882D83160313762D4E
:100B100003130317F82C6430C50003132F23831627
:100B200086178312861F952D972403172A10AA145F
:100B3000AA11AA1383160313E801E7017D08F60042
:100B40007C08F50083120317AB10031300348C1ECE
:100B5000A72D1808A9001A08F800A91CB12D181211
:100B60001816000000340317D2010408D1005210F7
:100B7000831B52144B0EF038CD00CD07E23ECE0061
:100B8000323ED0004B080F39CE07CE07D007E93EE2
:100B9000CF00CF07CF074A0E0F39CF07D007CF0DB1
:100BA000D00DD009D00D4A080F39D007CD0D073030
:100BB000CC000A30D007CF03031CDA2DCF07CE03B9
:100BC000031CDE2DCE07CD03031CE22DCD07CC0385
:100BD000031CE62D4C308400831707305105840731
:100BE0005030040203190C2E0008F700031DFE2DDF
:100BF000511A0A2ED119002E2030012E0830D100B2
:100C00003030F707770803130C1A082E0317032E4A
:100C100099000317840AF02D0008F7003030F70719
:100C2000770803130C1A162E0317112E990000349F
:100C30000317C803C9010313A72578080317CB00BE
:100C4000603C03182A2E4B087A3C031C2A2E4B08C2
:100C5000DF392B2E4B08CA004A08083C031D492ED9
:100C6000C9080319482EC9034A0803130C1A3A2E5F
:100C70000317352E990020300C1E3C2E99000317C7
:100C80004A0803130C1A462E0317412E9900031726
:100C9000662E4A081F3C0318662E4A087E3C031C39
:100CA000662E480849020318662E4908C90A4607F5
:100CB00084008313471883174A0880004A080313E7
:100CC0000C1A642E03175F2E990003174A080D3C77
:100CD000031D1B2E490846078400831347188317FA
:100CE0008001031300348C1E732E0317C701A0303C
:100CF000C6000630C8000313182600341030F70071
:100D0000FA010317D301D00CCF0C031C8D2E510810
:100D1000FA070318D30A5208D307D30CFA0CF90CBC
:100D2000F80CF70B832E03138A11BB2E0317C9018E
:100D3000CA01CC01CE01A030CD004D084E040319EC
:100D4000AA2E4C08CC0A4D07840083134E18831733
:100D50000008CB004B082F3C0318D22E4B08393C1F
